:1000000000308A002B280000A50A2708C83C2502DA
:1000100003190E28031C0E2885160F2885122808A0
:10002000C83C250203191828031C1828051519288F
:1000300005112908C83C250203192228031C22287F
:100040000516232805122508C73C031D2A28A501EB
:100050000130AA00682884011F3083051F1383160E
:100060001F109F101F119F110730831299008316D4
:100070000508831219088C11A501AB011F13831603
:100080001F109F101F119F1183121F10A001A01D90
:10009000512807308101813084000008C0390F38B1
:1000A00080006400813084000008C0392004800092
:1000B0009001703083168F048C0102308500811707
:1000C0009601950183128B018C018501A6010428FC
:1000D000A608031D59290630A6002B08003A03196B
:1000E000B428013A0319BA28033A0319C228013A7D
:1000F0000319CA28073A0319CF28013A0319D72848
:10010000033A0319DC28013A0319E4280F3A0319CA
:10011000EC28013A0319F428033A0319FC28013AA0
:1001200003190129073A03190929013A03190E296C
:10013000033A03191629013A03191E291F3A031914
:100140002629013A03192E29033A03193329013AC2
:1001500003193B29073A03194029013A0319482991
:10016000033A031950295829A701A801A901013010
:10017000AB005929A90A2908C73C031DC128023030
:10018000AB005929A80A2808C73C031DC928033019
:10019000AB005929A90BCE280430AB005929A70A76
:1001A0002708C73C031DD6280530AB005929A80BEA
:1001B000DB280630AB005929A90A2908C73C031DD2
:1001C000E3280730AB005929A80A2808C73C031DBB
:1001D000EB280830AB005929A703A903A708031D82
:1001E000F3280930AB005929A70A2708C73C031D8B
:1001F000FB280A30AB005929A80B00290B30AB00B3
:100200005929A90A2908C73C031D08290C30AB004D
:100210005929A70B0D290D30AB005929A80A280828
:10022000C73C031D15290E30AB005929A70A270822
:10023000C73C031D1D290F30AB005929A803A90392
:10024000A808031D25291030AB005929A90A29083F
:10025000C73C031D2D291130AB005929A70B3229AA
:100260001230AB005929A80A2808C73C031D3A29B7
:100270001330AB005929A90B3F291430AB00592981
:10028000A70A2708C73C031D47291530AB00592989
:10029000A90A2908C73C031D4F291630AB0059296C
:1002A000A703A803A708031D57290230AB0059294B
:1002B0005929AA0803195E29AA01A6036728630021
:02400E00A430DC
:00000001FF
